:100000002500840A070A170A2C0A670A730AFC0CDF
:10001000060046060D0A000C0E0A010C000D4307EF
:10002000160A0C058C05FC0C06000605A30A09023D
:10003000A9023C0C890003072B0A69000A02AA02E4
:100040003C0C8A0003072B0A6A000B02AB02180C57
:100050008B0003066B00A50A0C02400E000D430640
:10006000660A0C02200E000D43074F0A080C8B0095
:100070004307410A2A024307410A8C05FC0C06008B
:100080000605080C8B0043074F0A010C8A00430742
:100090004F0AFC0C06000604AC05EF0C6C01130CB7
:1000A0008B0043075A0A2A0243075A0A8C05FC0CA4
:1000B00006000605160C8B004307660A2A02430752
:1000C000660AFC0C06000604EF0C6C01A60A0F027F
:1000D0004306720A700A00000000000000000000E1
:1000E000EF026B0AB70A0C02010E000D4306830AE9
:1000F000080C2B006A006900CC05DF0C6C01FE0CBB
:100100006C01050C2D00BC0A6400040C2700670775
:100110008D0A070C61000F0C0200040007020200A8
:10012000FC0C06000604FC0C060026056C00010C05
:100130002D006E006100120C2B006A0069000102A4
:100140004306A40A020A9F0A030A040A0C02100EBC
:10015000000D4307BB0A0E02AE020D028E004307DC
:10016000BB0AFC0C06002604640C2F00050AFC0CDC
:0C017000060026056E00060A9F0A030028
:021FFE00D80FFA
:00000001FF
